:020000040800F2
:1000000000060020E1020008E3020008E302000805
:10001000E3020008E3020008E3020008E30200082C
:10002000E3020008E3020008E3020008ED340008E0
:10003000E3020008E3020008E3020008E30200080C
:10004000E3020008E3020008E3020008E3020008FC
:10005000E3020008E3020008D5380008013900086F
:100060002D3900085939000885390008E3020008D5
:10007000E3020008E3020008E3020008E3020008CC
:10008000E3020008E3020008E3020008E3020008BC
:10009000E3020008E3020008E3020008B1390008A7
:1000A000E3020008E3020008E3020008E30200089C
:1000B000E3020008E3020008E3020008E30200088C
:1000C000E3020008E3020008E3020008E30200087C
:1000D000E3020008E3020008E3020008E30200086C
:1000E000153A0008E3020008E3020008E3020008F2
:1000F000E3020008E3020008E3020008E30200084C
:10010000E3020008E3020008893A0008E30200085D
:10011000E3020008E3020008E3020008E30200082B
:10012000E3020008E3020008E3020008E30200081B
:10013000E3020008E3020008E3020008E30200080B
:10014000E3020008E3020008E3020008E3020008FB
:10015000E3020008E3020008E3020008E3020008EB
:10016000E3020008E3020008E3020008E3020008DB
:10017000E30200086D2E0008E3020008E302000815
:10018000E3020008E3020008E3020008E3020008BB
:10019000E3020008E3020008E3020008E3020008AB
:1001A000E3020008E3020008E3020008E30200089B
:1001B000E3020008E3020008E3020008E30200088B
:1001C000E3020008E3020008E3020008E30200087B
:1001D000E3020008592E0008E3020008E3020008C9
:1001E000E3020008E3020008E3020008E30200085B
:1001F000E3020008E3020008E3020008E30200084B
:10020000E3020008E3020008E3020008E30200083A
:10021000E3020008E3020008E3020008E30200082A
:10022000E3020008E3020008E3020008E30200081A
:10023000E3020008E3020008E3020008E30200080A
:10024000E3020008E3020008E3020008E3020008FA
:10025000E3020008E3020008E3020008E3020008EA
:10026000E3020008E3020008E3020008E3020008DA
:10027000E3020008E3020008E3020008E3020008CA
:10028000E3020008E3020008E3020008E3020008BA
:10029000E3020008E3020008E3020008E3020008AA
:1002A000E3020008E3020008E3020008E30200089A
:1002B000E3020008E3020008E3020008E30200088A
:1002C000E3020008E3020008E3020008E30200087A
:1002D000E3020008E3020008E3020008E30200086A
:1002E00002E000F000F8FEE772B6374880F30888B5
:1002F000364880F3098836483649086040F20000E5
:10030000CCF200004EF63471CEF200010860BFF36B
:100310004F8FBFF36F8F40F20000C0F2F0004EF637
:100320008851CEF200010860BFF34F8FBFF36F8F8B
:100330004FF00000E1EE100A4EF63C71CEF20001E3
:100340000860062080F31488BFF36F8F01F0FAFF76
:1003500003F01EF84FF055301F491B4A91423CBF35
:1003600041F8040BFAE71D49184A91423CBF41F895
:10037000040BFAE71A491B4A1B4B9A423EBF51F83D
:10038000040B42F8040BF8E700201849184A914280
:100390003CBF41F8040BFAE702F012F803F07CF8D6
:1003A000144C154DAC4203DA54F8041B8847F9E7A6
:1003B00000F042F8114C124DAC4203DA54F8041B21
:1003C0008847F9E701F0FABF00060020002200206C
:1003D0000000000808ED00E00000002000060020FA
:1003E000683E0008002200205C22002060220020DD
:1003F00034430020E0020008E0020008E0020008A8
:10040000E00200082DE9F04F2DED108AC1F80CD064
:10041000D0F80CD0BDEC108ABDE8F08F002383F338
:1004200011882846A047002001F0FEFAFEE701F0FF
:1004300067FA00DFFEE7000038B501F043FF05462C
:1004400001F076FF0446D0B90F4B9D4219D001331D
:100450009D4241F2883512BF044600250124002048
:1004600001F03AFF0CB100F077F800F053FD00F016
:1004700005FC284600F010F900F06EF8F9E70025B9
:10048000EDE70546EBE700BF010007B008B500F057
:10049000C7FBA0F120035842584108BD07B541F2FF
:1004A0001203022101A8ADF8043000F0D7FB03B01D
:1004B0005DF804FB38B5302383F3118817480368CF
:1004C0000BB101F07DFB0023154A4FF47A711348FC
:1004D00001F06CFB002383F31188124C236813B1E5
:1004E0002368013B2360636813B16368013B636069
:1004F0000D4D2B7833B963687BB9022000F084FC82
:10050000322363602B78032B07D163682BB9022059
:1005100000F07AFC4FF47A73636038BD60220020EB
:10052000B50400088023002078220020084B1870B2
:1005300003280CD8DFE800F008050208022000F0CC
:1005400059BC022000F04EBC024B00225A6070479A
:100550007822002080230020F8B5494B494A1C46E8
:100560001968013100F08A8004339342F8D162683F
:10057000454B9A4240F28280444B9B6803F10063F2
:1005800003F500339A4279D2002000F09DFB02204F
:10059000FFF7CCFF3E4B0021D3F8E820C3F8E8106A
:1005A000D3F81021C3F81011D3F81021D3F8EC20A0
:1005B000C3F8EC10D3F81421C3F81411D3F81421A4
:1005C000D3F8F020C3F8F010D3F81821C3F81811AD
:1005D000D3F81821D3F8802042F00072C3F88020AD
:1005E000D3F8802022F00072C3F88020D3F8803046
:1005F00072B64FF0E023C3F8084DD4E90004BFF30E
:100600004F8FBFF36F8F234AC2F88410BFF34F8F11
:10061000536923F480335361BFF34F8FD2F8803096
:1006200043F6E076C3F3C905C3F34E335B0103EA37
:10063000060C29464CEA81770139C2F87472F9D266
:10064000203B13F1200FF2D1BFF34F8FBFF36F8F19
:10065000BFF34F8FBFF36F8F536923F400335361A0
:100660000023C2F85032BFF34F8FBFF36F8F302398
:1006700083F31188854680F308882047F8BD00BFC2
:100680000000020820000208FFFF010800220020ED
:100690000044025800ED00E02DE9F04F93B0B44B58
:1006A0002022FF2100900AA89D6800F0DDFBB14ADE
:1006B0001378A3B90121B04811700360302383F38C
:1006C000118803680BB101F07BFA0023AB4A4FF4A9
:1006D0007A71A94801F06AFA002383F31188009B1C
:1006E00013B1A74B009A1A60A64A1378032B03D0C4
:1006F00000231370A24A53604FF0000A009CD346B7
:100700005646D146012000F075FB24B19C4B1B6876
:10071000002B00F02682002000F082FA0390039B59
:10072000002BF2DB012000F05DFB039B213B1F2B24
:10073000E8D801A252F823F0B9070008E107000841
:1007400075080008050700080507000805070008E8
:1007500007090008D70A0008F1090008530A000831
:100760007B0A0008A10A000805070008B30A000870
:1007700005070008250B00085908000805070008B0
:10078000690B0008C507000859080008050700089C
:10079000530A0008050700080507000805070008B8
:1007A00005070008050700080507000805070008F9
:1007B00005070008750800080220FFF767FE0028FB
:1007C00040F0F981009B022105A8BAF1000F08BF93
:1007D0001C4641F21233ADF8143000F03FFA91E7B5
:1007E0004FF47A7000F01CFA071EEBDB0220FFF7D3
:1007F0004DFE0028E6D0013F052F00F2DE81DFE844
:1008000007F0030A0D1013360523042105A80593EC
:1008100000F024FA17E004215548F9E704215A486A
:10082000F6E704215948F3E74FF01C08404608F169
:10083000040800F04BFA0421059005A800F00EFA18
:10084000B8F12C0FF2D101204FF0000900FA07F7A0
:1008500047EA0B0B5FFA8BFB00F052FB26B10BF063
:100860000B030B2B08BF0024FFF718FE4AE70421F7
:100870004748CDE7002EA5D00BF00B030B2BA1D1E1
:100880000220FFF703FE074600289BD00120002628
:1008900000F01AFA0220FFF749FE5FFA86F8404698
:1008A00000F022FA0446B0B1039940460136A1F1A6
:1008B00040025142514100F027FA0028EDD1BA46DA
:1008C000044641F21213022105A83E46ADF8143049
:1008D00000F0C4F916E725460120FFF727FE244B58
:1008E0009B68AB4207D9284600F0F0F9013040F090
:1008F00067810435F3E70025224BBA463E461D705A
:100900001F4B5D60A8E7002E3FF45CAF0BF00B03BC
:100910000B2B7FF457AF0220FFF708FE322000F0C8
:100920007FF9B0F10008FFF64DAF18F003077FF430
:1009300049AF0F4A08EB0503926893423FF642AF76
:10094000B8F5807F3FF73EAF124BB845019323DDEA
:100950004FF47A7000F064F90390039A002AFFF6CE
:1009600031AF039A0137019B03F8012BEDE700BF7C
:10097000002200207C23002060220020B504000813
:10098000802300207822002004220020082200205A
:100990000C2200207C220020C820FFF777FD0746AC
:1009A00000283FF40FAF1F2D11D8C5F120020AAB6C
:1009B00025F0030084494245184428BF424601926D
:1009C00000F02CFA019AFF217F4800F04DFA4FEA1F
:1009D000A803C8F387027C492846019300F04CFA2B
:1009E000064600283FF46DAF019B05EB830533E716
:1009F0000220FFF74BFD00283FF4E4AE00F0A2F91F
:100A000000283FF4DFAE0027B846704B9B68BB421E
:100A100018D91F2F11D80A9B01330ED027F00303DA
:100A200012AA134453F8203C05934046042205A91A
:100A3000043700F09BFA8046E7E7384600F046F9B5
:100A40000590F2E7CDF81480042105A800F006F91E
:100A500002E70023642104A8049300F0F5F80028BD
:100A60007FF4B0AE0220FFF711FD00283FF4AAAEDC
:100A7000049800F05DF90590E6E70023642104A8DE
:100A8000049300F0E1F800287FF49CAE0220FFF709
:100A9000FDFC00283FF496AE049800F04BF9EAE71D
:100AA0000220FFF7F3FC00283FF48CAE00F05AF967
:100AB000E1E70220FFF7EAFC00283FF483AE05A936
:100AC000142000F055F907460421049004A800F012
:100AD000C5F83946B9E7322000F0A2F8071EFFF644
:100AE00071AEBB077FF46EAE384A07EB090392681C
:100AF00093423FF667AE0220FFF7C8FC00283FF4A0
:100B000061AE27F003074F44B9453FF4A5AE484610
:100B100009F1040900F0DAF80421059005A800F0B5
:100B20009DF8F1E74FF47A70FFF7B0FC00283FF42E
:100B300049AE00F007F9002844D00A9B01330BD0DE
:100B400008220AA9002000F097F900283AD02022B4
:100B5000FF210AA800F088F9FFF7A0FC1C4800F06C
:100B600069FF13B0BDE8F08F002E3FF42BAE0BF001
:100B70000B030B2B7FF426AE0023642105A80593FD
:100B800000F062F8074600287FF41CAE0220FFF751
:100B90007DFC804600283FF415AEFFF77FFC41F254
:100BA000883000F047FF059800F0DEF946463C46E5
:100BB00000F0A6F9A6E506464EE64FF0000901E66C
:100BC000BA467EE637467CE67C22002000220020E2
:100BD000A08601000F4B70B51B780C460133DBB2C9
:100BE000012B11D80C4D4FF47A732968A2FB033204
:100BF00022460E6A01462846B047844204D1074B7C
:100C0000002201201A7070BD4FF4FA7000F012FF3C
:100C10000020F8E71022002028260020B42300201E
:100C2000002307B5024601210DF107008DF80730BA
:100C3000FFF7D0FF20B19DF8070003B05DF804FB7B
:100C40004FF0FF30F9E700000A46042108B5FFF72E
:100C5000C1FF80F00100C0B2404208BD30B4054C75
:100C60000A46014623682046DD69034BAC4630BC8A
:100C7000604700BF28260020A086010070B5104CF8
:100C80000025104E01F0F6F9208030682388834259
:100C90000CD800252088013801F0E8F923880544A4
:100CA000013BB5F5802F2380F4D370BD01F0DEF950
:100CB000336805440133B5F5003F3360E5D3E8E719
:100CC000B62300208823002001F0B2BA00F10060B2
:100CD00000F500300068704700F10060920000F5F8
:100CE000003001F029BA0000054B1A68054B1B883B
:100CF0009B1A834202D9104401F0B8B90020704712
:100D000088230020B623002038B50446074D29B1BA
:100D100028682044BDE8384001F0C0B92868204464
:100D200001F0AAF90028F3D038BD00BF88230020C5
:100D30000020704700F1FF5000F58F10D0F8000838
:100D400070470000064991F8243033B1002308228F
:100D5000086A81F82430FFF7BFBF0120704700BF49
:100D60008C230020014B1868704700BF0010005C06
:100D7000194B01380322084470B51D68174BC5F3A1
:100D80000B042D0C1E88A6420BD15C680A46013C60
:100D9000824213460FD214F9016F4EB102F8016B73
:100DA000F6E7013A03F10803ECD181420B4602D287
:100DB0002C2203F8012B0424094A1688AE4204D1E0
:100DC000984284BF967803F8016B013C02F104025B
:100DD000F3D1581A70BD00BF0010005C142200202F
:100DE000803B0008022802D1014B04229A6170471F
:100DF00000080258022803D1024B4FF480229A6166
:100E0000704700BF00080258022804D1024A536903
:100E100083F004035361704700080258002310B5A3
:100E2000934203D0CC5CC4540133F9E710BD0000F9
:100E3000013810B510F9013F3BB191F900409C42D7
:100E400003D11AB10131013AF4E71AB191F9002046
:100E5000981A10BD1046FCE703460246D01A12F954
:100E6000011B0029FAD1704702440346934202D085
:100E700003F8011BFAE770472DE9F8431F4D1446AC
:100E80000746884695F8242052BBDFF870909CB343
:100E900095F824302BB92022FF2148462F62FFF716
:100EA000E3FF95F824004146C0F1080205EB8000FD
:100EB000A24228BF2246D6B29200FFF7AFFF95F8B4
:100EC0002430A41B17441E449044E4B2F6B2082E0A
:100ED00085F82460DBD1FFF735FF0028D7D108E083
:100EE0002B6A03EB82038342CFD0FFF72BFF00284E
:100EF000CBD10020BDE8F8830120FBE78C23002044
:100F0000024B1A78024B1A70704700BFB4230020BE
:100F10001022002010B5104C104800F0B9F82146FE
:100F20000E4800F0E1F824680D48D4F89020D2F87B
:100F3000043843F00203C2F8043800F07BFD09498D
:100F4000204600F0DFF9D4F89020D2F8043823F0DE
:100F50000203C2F8043810BD3C3C000828260020DB
:100F600040420F00443C00087047000030B50A447E
:100F7000084D91420DD011F8013B5840082340F331
:100F80000004013B2C4013F0FF0384EA5000F6D12B
:100F9000EFE730BD2083B8ED02684368114301607C
:100FA00003B118477047000013B5406B00F580543B
:100FB000D4F8A4381A681178042914D1017C0229C4
:100FC00011D11979012312898B4013420BD101A948
:100FD0004C3002F093F8D4F8A4480246019B2179E2
:100FE000206800F0DFF902B010BD0000143002F0FC
:100FF00015B800004FF0FF33143002F00FB80000B6
:101000004C3002F0E7B800004FF0FF334C3002F0F4
:10101000E1B80000143001F0E3BF00004FF0FF31F1
:10102000143001F0DDBF00004C3002F0B3B8000016
:101030004FF0FF324C3002F0ADB800000020704796
:1010400010B500F58054D4F8A4381A681178042932
:1010500017D1017C022914D15979012352898B407F
:1010600013420ED1143001F075FF024648B1D4F896
:10107000A4484FF4407361792068BDE8104000F047
:101080007FB910BD406BFFF7DBBF00007047000069
:101090007FB5124B01250426044603600023057426
:1010A00000F1840243602946C0E902330C4B0290F0
:1010B000143001934FF44073009601F027FF094B61
:1010C00004F69442294604F14C000294CDE90063F1
:1010D0004FF4407301F0EEFF04B070BD903B000888
:1010E00085100008A90F00080A68302383F31188CF
:1010F0000B790B3342F823004B79133342F823006A
:101100008B7913B10B3342F8230000F58053C3F8F9
:10111000A41802230374002080F311887047000094
:1011200038B5037F044613B190F85430ABB90125AC
:10113000201D0221FFF730FF04F114006FF00101C0
:10114000257700F09FFC04F14C0084F854506FF0B8
:101150000101BDE8384000F095BC38BD10B5012153
:1011600004460430FFF718FF0023237784F8543037
:1011700010BD000038B504460025143001F0DEFE35
:1011800004F14C00257701F0ADFF201D84F8545088
:101190000121FFF701FF2046BDE83840FFF750BFAF
:1011A00090F8803003F06003202B06D190F8812066
:1011B0000023212A03D81F2A06D800207047222A9C
:1011C000FBD1C0E91D3303E0034A4267072282676F
:1011D000C3670120704700BF2C22002037B500F5FF
:1011E0008055D5F8A4381A68117804291AD1017CE1
:1011F000022917D11979012312898B40134211D189
:1012000000F14C04204602F02DF858B101A9204607
:1012100001F074FFD5F8A4480246019B21792068AB
:1012200000F0C0F803B030BD01F10B03F0B550F889
:10123000236085B004460D46FEB1302383F3118848
:1012400004EB8507301D0821FFF7A6FEFB6806F1B9
:101250004C005B691B681BB1019001F05DFF0198B8
:1012600003A901F04BFF024648B1039B29462046E3
:1012700000F098F8002383F3118805B0F0BDFB68F7
:101280005A691268002AF5D01B8A013B1340F1D13C
:1012900004F18002EAE70000133138B550F821402C
:1012A000ECB1302383F3118804F58053D3F8A428DC
:1012B0001368527903EB8203DB689B695D6845B173
:1012C00004216018FFF768FE294604F1140001F0BC
:1012D0004BFE2046FFF7B4FE002383F3118838BD90
:1012E0007047000001F002B901234022002110B52F
:1012F000044600F8303BFFF7B7FD0023C4E9013393
:1013000010BD000010B53023044683F31188242259
:10131000416000210C30FFF7A7FD204601F008F9DD
:1013200002230020237080F3118810BD70B500EBFC
:101330008103054650690E461446DA6018B1102242
:101340000021FFF791FDA06918B110220021FFF7DD
:101350008BFD31462846BDE8704001F0EFB9000032
:1013600083682022002103F0011310B50446836036
:101370001030FFF779FD2046BDE8104001F06ABA51
:10138000F0B4012500EB810447898D40E4683D43BA
:10139000A469458123600023A2606360F0BC01F072
:1013A00087BA0000F0B4012500EB810407898D4065
:1013B000E4683D436469058123600023A2606360A3
:1013C000F0BC01F0FDBA000070B502230025044610
:1013D000242203702946C0F888500C3040F8045C81
:1013E000FFF742FD204684F8705001F03BF9636836
:1013F0001B6823B129462046BDE87040184770BDE0
:101400000378052B10B504460AD080F88C300523EC
:10141000037043681B680BB1042198470023A36045
:1014200010BD00000178052906D190F88C20436892
:1014300002701B6803B118477047000070B590F840
:101440007030044613B1002380F8703004F180023C
:10145000204601F023FA63689B68B3B994F88030A2
:1014600013F0600535D00021204601F015FD002164
:10147000204601F005FD63681B6813B10621204674
:101480009847062384F8703070BD2046984700289E
:10149000E4D0B4F88630A26F9A4288BFA36794F96B
:1014A0008030A56F002B4FF0300380F20381002DB8
:1014B00000F0F280092284F8702083F31188002163
:1014C0002046D4E91D23FFF76DFF002383F3118825
:1014D000DAE794F8812003F07F0343EA022340F225
:1014E0000232934200F0C58021D8B3F5807F48D006
:1014F0000DD8012B3FD0022B00F09380002BB2D1EE
:1015000004F1880262670222A267E367C1E7B3F5CC
:10151000817F00F09B80B3F5407FA4D194F88230A6
:10152000012BA0D1B4F8883043F0020332E0B3F5C8
:10153000006F4DD017D8B3F5A06F31D0A3F5C063BD
:10154000012B90D86368204694F882205E6894F856
:101550008310B4F88430B047002884D043686367B0
:101560000368A3671AE0B3F5106F36D040F6024265
:1015700093427FF478AF5C4B63670223A367002339
:10158000C3E794F88230012B7FF46DAFB4F8883054
:1015900023F00203A4F88830C4E91D55E56778E715
:1015A000B4F88030B3F5A06F0ED194F882302046A5
:1015B00084F88A3001F0B4F863681B6813B1012124
:1015C00020469847032323700023C4E91D339CE77A
:1015D00004F18B0363670123C3E72378042B10D145
:1015E000302383F311882046FFF7BAFE85F3118874
:1015F0000321636884F88B5021701B680BB120466F
:10160000984794F88230002BDED084F88B30042386
:10161000237063681B68002BD6D0022120469847B0
:10162000D2E794F8843020461D0603F00F010AD556
:1016300001F026F9012804D002287FF414AF2B4BC7
:101640009AE72B4B98E701F00DF9F3E794F8823015
:10165000002B7FF408AF94F8843013F00F01B3D05F
:101660001A06204602D501F02FFCADE701F020FC60
:10167000AAE794F88230002B7FF4F5AE94F884301A
:1016800013F00F01A0D01B06204602D501F004FC88
:101690009AE701F0F5FB97E7142284F8702083F3B2
:1016A00011882B462A4629462046FFF769FE85F316
:1016B0001188E9E65DB1152284F8702083F3118862
:1016C00000212046D4E91D23FFF75AFEFDE60B2238
:1016D00084F8702083F311882B462A462946204639
:1016E000FFF760FEE3E700BFC03B0008B83B00081F
:1016F000BC3B000838B590F870300446002B3ED053
:10170000063BDAB20F2A34D80F2B32D8DFE803F0C9
:1017100037313108223231313131313131313737DE
:10172000856FB0F886309D4214D2C3681B8AB5FB22
:10173000F3F203FB12556DB9302383F311882B4666
:101740002A462946FFF72EFE85F311880A2384F8DE
:1017500070300EE0142384F87030302383F3118846
:10176000002320461A461946FFF70AFE002383F39A
:10177000118838BDC36F03B198470023E7E7002104
:10178000204601F089FB0021204601F079FB6368C7
:101790001B6813B10621204698470623D7E70000AF
:1017A00010B590F870300446142B29D017D8062BAA
:1017B00005D001D81BB110BD093B022BFBD800217D
:1017C000204601F069FB0021204601F059FB6368C7
:1017D0001B6813B1062120469847062319E0152BF4
:1017E000E9D10B2380F87030302383F31188002374
:1017F0001A461946FFF7D6FD002383F31188DAE76E
:10180000C3689B695B68002BD5D1C36F03B1984750
:10181000002384F87030CEE70023826803750369E3
:101820001B6899689142FBD25A680360426010605D
:101830005860704700238268037503691B689968C4
:101840009142FBD85A68036042601060586070474C
:1018500008B50846302383F311880B7D032B05D090
:10186000042B0DD02BB983F3118808BD8B6900229E
:101870001A604FF0FF338361FFF7CEFF0023F2E7DA
:10188000D1E9003213605A60F3E70000FFF7C4BFEC
:10189000054BD96808751868026853601A60012200
:1018A000D8600275FEF7AEBDB82300200C4B30B5F2
:1018B000DD684B1C87B004460FD02B46094A6846AA
:1018C00000F074F92046FFF7E3FF009B13B1684670
:1018D00000F076F9A86907B030BDFFF7D9FFF9E746
:1018E000B823002051180008044B1A68DB68906880
:1018F0009B68984294BF002001207047B8230020C5
:10190000084B10B51C68D868226853601A60012221
:10191000DC602275FFF78EFF01462046BDE81040CF
:10192000FEF770BDB8230020044B1A68DB6892688C
:101930009B689A4201D9FFF7E3BF7047B8230020A4
:1019400038B5074C01230025064907482370656018
:1019500001F0C6FC0223237085F3118838BD00BF57
:1019600020260020C83B0008B823002000F05EB904
:10197000EFF3118020B9EFF30583302282F3118851
:101980007047000010B530B9EFF30584C4F30804C4
:1019900014B180F3118810BDFFF7C6FF84F31188DE
:1019A000F9E70000034A516853685B1A9842FBD874
:1019B000704700BF001000E08B60022308610846FA
:1019C0008B8270478368A3F1840243F8142C026968
:1019D00043F8442C426943F8402C094A43F8242C2C
:1019E000C268A3F1200043F8182C022203F80C2C43
:1019F000002203F80B2C034A43F8102C704700BF59
:101A00001D040008B823002008B5FFF7DBFFBDE880
:101A10000840FFF73BBF0000024BDB6898610F20D6
:101A2000FFF736BFB8230020302383F31188FFF778
:101A3000F3BF000008B50146302383F31188082066
:101A4000FFF734FF002383F3118808BD064BDB68E2
:101A500039B1426818605A60136043600420FFF790
:101A600025BF4FF0FF307047B8230020036898422D
:101A700006D01A680260506018469961FFF706BFE9
:101A80007047000038B504460D462068844200D1F6
:101A900038BD036823605C608561FFF7F7FEF4E7FB
:101AA000036810B59C68A2420CD85C688A600B6021
:101AB0004C602160596099688A1A9A604FF0FF3330
:101AC000836010BD121B1B68ECE700000A2938BFB9
:101AD0000A2170B504460D460A26601901F0F8FB8C
:101AE00001F0E0FB041BA54203D8751C04462E46FA
:101AF000F3E70A2E04D90120BDE8704001F030BCA4
:101B000070BD0000F8B5144B0D460A2A4FF00A07C5
:101B1000D96103F11001826038BF0A22416019695E
:101B20001446016048601861A81801F0C1FB01F07B
:101B3000B9FB431B0646A34206D37C1C2819274643
:101B4000354601F0C5FBF2E70A2F04D90120BDE8B4
:101B5000F84001F005BCF8BDB8230020F8B50646F2
:101B60000D4601F09FFB0F4A134653F8107F9F422A
:101B700006D12A4601463046BDE8F840FFF7C2BF0D
:101B8000D169BB68441A2C1928BF2C46A34202D93C
:101B90002946FFF79BFF224631460348BDE8F8403F
:101BA000FFF77EBFB8230020C8230020C0E903232D
:101BB000002310B45DF8044B4361FFF7CFBF000072
:101BC00010B5194C236998420DD08168D0E90032D4
:101BD00013605A609A680A449A60002303604FF0C9
:101BE000FF33A36110BD0268234643F8102F5360F2
:101BF0000022026022699A4203D1BDE8104001F040
:101C000061BB936881680B44936001F04BFB2269D0
:101C1000E1699268441AA242E4D91144BDE8104037
:101C2000091AFFF753BF00BFB82300202DE9F04782
:101C3000DFF8BC8008F110072C4ED8F8105001F0E6
:101C400031FBD8F81C40AA68031B9A423ED81444C2
:101C50004FF00009D5E90032C8F81C4013605A6003
:101C6000C5F80090D8F81030B34201D101F02AFB3A
:101C700089F31188D5E9033128469847302383F347
:101C800011886B69002BD8D001F00CFB6A69A0EBBE
:101C9000040982464A450DD2022001F061FB002270
:101CA000D8F81030B34208D151462846BDE8F04775
:101CB000FFF728BF121A2244F2E712EB090929465E
:101CC000384638BF4A46FFF7EBFEB5E7D8F8103084
:101CD000B34208D01444C8F81C00211AA960BDE81A
:101CE000F047FFF7F3BEBDE8F08700BFC823002030
:101CF000B823002000207047FEE700007047000076
:101D00004FF0FF307047000002290CD0032904D0A7
:101D10000129074818BF00207047032A05D8054845
:101D200000EBC2007047044870470020704700BFB6
:101D3000A03C00083C220020543C000870B59AB03A
:101D400005460846144601A900F0C2F801A8FFF7AD
:101D500083F8431C0022C6B25B001046C5E900347C
:101D600023700323023404F8013C01ABD1B20234E6
:101D70008E4201D81AB070BD13F8011B013204F86D
:101D8000010C04F8021CF1E708B5302383F3118835
:101D90000348FFF723FA002383F3118808BD00BF2F
:101DA0002826002090F8803003F01F02012A07D176
:101DB00090F881200B2A03D10023C0E91D3315E0E0
:101DC00003F06003202B08D1B0F884302BB990F8D1
:101DD0008120212A03D81F2A04D8FFF7E1B9222A3B
:101DE000EBD0FAE7034A426707228267C367012004
:101DF000704700BF3322002007B5052917D8DFE858
:101E000001F0191603191920302383F31188104AA1
:101E100001210190FFF78AFA019802210D4AFFF78C
:101E200085FA0D48FFF7A6F9002383F3118803B064
:101E30005DF804FB302383F311880748FFF770F93E
:101E4000F2E7302383F311880348FFF787F9EBE7C4
:101E5000F43B0008183C00082826002038B50C4D3B
:101E60000C4C2A460C4904F10800FFF767FF05F106
:101E7000CA0204F110000949FFF760FF05F5CA72B4
:101E800004F118000649BDE83840FFF757BF00BF0E
:101E9000003F00203C220020D43B0008DE3B00082D
:101EA000E93B000870B5044608460D46FEF7D4FF2E
:101EB000C6B22046013403780BB9184670BD3246CD
:101EC0002946FEF7B5FF0028F3D10120F6E7000010
:101ED0002DE9F84F05460C46FEF7BEFF2D49C6B268
:101EE0002846FFF7DFFF08B10436F6B22A49284634
:101EF000FFF7D8FF08B11036F6B2632E0DD8DFF821
:101F00009490DFF894A0DFF89C80DFF89CB0234F1A
:101F10002E7846B92670BDE8F88F29462046BDE8E0
:101F2000F84F01F00FBE252E30D107224946284632
:101F3000FEF77EFF70B93B6807350B3444F80B3C65
:101F40007B6844F8073C3B8924F8033CBB7A04F8DF
:101F5000013CDDE7082251462846FEF769FFA8B993
:101F6000A21C0F4B19780232090911F8081002F867
:101F7000041C13F8011B01F00F015B4511F8081058
:101F800002F8031CEED118340835C1E7013504F816
:101F9000016BBDE7C03C0008E93B0008C83C0008F5
:101FA00000E8F11FD43C00080CE8F11FBFF34F8F8D
:101FB000044B1A695107FCD1D3F810215207F8D10C
:101FC000704700BF0020005208B50D4B1B78ABB91D
:101FD000FFF7ECFF0B4BDA68D10704D50A4A5A60C9
:101FE00002F188325A60D3F80C21D20706D5064A8E
:101FF000C3F8042102F18832C3F8042108BD00BFF0
:102000005E410020002000522301674508B5114BB6
:102010001B78F3B9104B1A69510703D5DA6842F0FF
:102020004002DA60D3F81021520705D5D3F80C210D
:1020300042F04002C3F80C21FFF7B8FF064BDA6804
:1020400042F00102DA60D3F80C2142F00102C3F839
:102050000C2108BD5E410020002000520F289ABFCD
:1020600000F5806040040020704700004FF400300D
:1020700070470000102070470F2808B50BD8FFF7F5
:10208000EDFF00F500330268013204D104308342D1
:10209000F9D1012008BD0020FCE700000F2870B531
:1020A000054645D8FFF764FC224CFFF77FFF064644
:1020B000FFF78AFF4FF0FF33072D6361C4F8143137
:1020C00020D82361FFF772FF2B0243F02403E36063
:1020D000E36843F08003E36023695A07FCD4284691
:1020E000FFF764FF4FF40031FFF7B8FF00F002F98B
:1020F0003046FFF78BFFFFF745FC2846BDE87040F0
:10210000FFF7BABFC4F81031FFF750FFA5F108037D
:102110001B0243F02403C4F80C31D4F80C3143F013
:102120008003C4F80C31D4F810315B07FBD4D6E738
:10213000002070BD002000522DE9F84F40EA020354
:1021400005460C461746D80602D00020BDE8F88F99
:1021500027F01F07DFF8D4B0FFF736FF2744BC4253
:1021600003D10120FFF752FFF0E720222946204645
:1021700001F0D8FC10B920352034F0E72B4605F1EA
:1021800020021E68711CE0D104339A42F9D1FFF796
:10219000EFFB05F17843234AB3F5801F224B28BF9C
:1021A0009A4603F1040338BF9046A2F1080228BF03
:1021B0009846A3F108033ABF9146DA469946FFF7DD
:1021C000F5FEC8F80060A5EB040CD9F8002004F176
:1021D0001C0142F00202C9F80020221FDAF8006058
:1021E00016F00506FAD152F8043F8A424CF8023044
:1021F000F4D1BFF34F8FFFF7D9FE4FF0FF32C8F88D
:102200000020D9F8002022F00202C9F80020FFF7D0
:10221000B9FB20222146284601F084FC0028AAD0E0
:1022200030469FE714200052102100521020005227
:1022300010B5084C237828B11BB9FFF7C5FE012360
:10224000237010BD002BFCD02070BDE81040FFF7BC
:10225000DDBE00BF5E4100200244074BD2B210B584
:10226000904200D110BD441C00B253F8200041F848
:10227000040BE0B2F4E700BF504000580E4B30B5FD
:102280001C6F240405D41C6F1C671C6F44F40044AD
:102290001C670A4C02442368D2B243F48073236063
:1022A000074B904200D130BD441C51F8045B00B292
:1022B00043F82050E0B2F4E70044025800480258C6
:1022C0005040005807B5012201A90020FFF7C4FFC4
:1022D000019803B05DF804FB13B50446FFF7F2FF65
:1022E000A04205D0012201A900200194FFF7C6FFFA
:1022F00002B010BD0144BFF34F8F064B884204D398
:10230000BFF34F8FBFF36F8F7047C3F85C0220306D
:10231000F4E700BF00ED00E0034B1A681AB9034A66
:10232000D2F8D0241A607047604100200040025863
:1023300008B5FFF7F1FF024B1868C0F3806008BDD5
:102340006041002070B5BFF34F8FBFF36F8F1A4A03
:102350000021C2F85012BFF34F8FBFF36F8F536944
:1023600043F400335361BFF34F8FBFF36F8FC2F855
:102370008410BFF34F8FD2F8803043F6E074C3F37C
:10238000C900C3F34E335B0103EA0406014646EA83
:1023900081750139C2F86052F9D2203B13F1200F48
:1023A000F2D1BFF34F8F536943F480335361BFF3CE
:1023B0004F8FBFF36F8F70BD00ED00E0FEE70000B0
:1023C000214B2248224A70B5904237D3214BC11E7F
:1023D000DA1C121A22F003028B4238BF00220021BD
:1023E000FEF742FD1C4A0023C2F88430BFF34F8F32
:1023F000D2F8803043F6E074C3F3C900C3F34E3320
:102400005B0103EA0406014646EA81750139C2F818
:102410006C52F9D2203B13F1200FF2D1BFF34F8F52
:10242000BFF36F8FBFF34F8FBFF36F8F0023C2F8DF
:102430005032BFF34F8FBFF36F8F70BD53F8041B43
:1024400040F8041BC0E700BFC43E0008344300202E
:10245000344300203443002000ED00E0074BD3F864
:10246000D81021EA0001C3F8D810D3F8002122EADD
:102470000002C3F80021D3F800317047004402582D
:1024800070B5D0E9244300224FF0FF359E6804EB7D
:1024900042135101D3F80009002805DAD3F80009E6
:1024A00040F08040C3F80009D3F8000B002805DA9B
:1024B000D3F8000B40F08040C3F8000B01326318E2
:1024C0009642C3F80859C3F8085BE0D24FF00113F5
:1024D000C4F81C3870BD0000890141F02001016181
:1024E00003699B06FCD41220FFF75CBA10B50A4CB6
:1024F0002046FEF7F9FE094BC4F89030084BC4F8AB
:102500009430084C2046FEF7EFFE074BC4F890309D
:10251000064BC4F8943010BD644100200000084010
:102520000C3D00080042002000000440183D000857
:1025300070B503780546012B5CD1434BD0F8904031
:10254000984258D1414B0E216520D3F8D82042F053
:102550000062C3F8D820D3F8002142F00062C3F82B
:102560000021D3F80021D3F8802042F00062C3F8A4
:102570008020D3F8802022F00062C3F88020D3F8B6
:10258000803000F0ADFC324BE360324BC4F80038D1
:102590000023D5F89060C4F8003EC02323604FF4B8
:1025A0000413A3633369002BFCDA01230C2033618D
:1025B000FFF7F8F93369DB07FCD41220FFF7F2F9D3
:1025C0003369002BFCDA00262846A660FFF758FF87
:1025D0006B68C4F81068DB68C4F81468C4F81C6839
:1025E00083BB1D4BA3614FF0FF336361A36843F0CE
:1025F0000103A36070BD194B9842C9D1134B4FF032
:102600008060D3F8D82042F00072C3F8D820D3F805
:10261000002142F00072C3F80021D3F80021D3F862
:10262000802042F00072C3F88020D3F8802022F08E
:102630000072C3F88020D3F88030FFF70FFF0E211F
:102640004D209EE7064BCDE7644100200044025830
:102650004014004003002002003C30C00042002033
:10266000083C30C0F8B5D0F89040054600214FF046
:1026700000662046FFF730FFD5F8941000234FF096
:1026800001128F684FF0FF30C4F83438C4F81C28AA
:1026900004EB431201339F42C2F80069C2F8006B99
:1026A000C2F80809C2F8080BF2D20B68D5F89020DE
:1026B000C5F89830636210231361166916F010068E
:1026C000FBD11220FFF76EF9D4F8003823F4FE6333
:1026D000C4F80038A36943F4402343F01003A36116
:1026E0000923C4F81038C4F814380B4BEB604FF0D2
:1026F000C043C4F8103B094BC4F8003BC4F8106950
:10270000C4F80039D5F8983003F1100243F480136F
:10271000C5F89820A362F8BDE83C0008408000108E
:10272000D0F8902090F88A10D2F8003823F4FE6395
:1027300043EA0113C2F80038704700002DE9F8435E
:1027400000EB8103D0F890500C468046DA680FFA0F
:1027500081F94801166806F00306731E022B05EB8B
:1027600041134FF0000194BFB604384EC3F8101B5C
:102770004FF0010104F1100398BF06F1805601FAF1
:1027800003F3916998BF06F5004600293AD0578AAD
:1027900004F15801374349016F50D5F81C180B4319
:1027A0000021C5F81C382B180127C3F81019A740C1
:1027B0005369611E9BB3138A928B9B08012A88BFC1
:1027C0005343D8F89820981842EA034301F1400295
:1027D0002146C8F89800284605EB82025360FFF7AF
:1027E0007BFE08EB8900C3681B8A43EA84534834A4
:1027F0001E4364012E51D5F81C381F43C5F81C78C0
:10280000BDE8F88305EB4917D7F8001B21F4004118
:10281000C7F8001BD5F81C1821EA0303C0E704F130
:102820003F030B4A2846214605EB83035A60FFF716
:1028300053FE05EB4910D0F8003923F40043C0F8EB
:102840000039D5F81C3823EA0707D7E700800010C5
:1028500000040002D0F894201268C0F89820FFF716
:102860000FBE00005831D0F8903049015B5813F486
:10287000004004D013F4001F0CBF02200120704759
:102880004831D0F8903049015B5813F4004004D02F
:1028900013F4001F0CBF02200120704700EB8101E0
:1028A000CB68196A0B6813604B685360704700006F
:1028B00000EB810330B5DD68AA691368D36019B9EC
:1028C000402B84BF402313606B8A1468D0F890209B
:1028D0001C4402EB4110013C09B2B4FBF3F4634326
:1028E000033323F0030343EAC44343F0C043C0F877
:1028F000103B2B6803F00303012B0ED1D2F80838EC
:1029000002EB411013F4807FD0F8003B14BF43F07A
:10291000805343F00053C0F8003B02EB4112D2F861
:10292000003B43F00443C2F8003B30BD2DE9F041C9
:10293000D0F8906005460C4606EB4113D3F8087BAF
:102940003A07C3F8087B08D5D6F814381B0704D516
:1029500000EB8103DB685B689847FA071FD5D6F860
:102960001438DB071BD505EB8403D968CCB98B6918
:10297000488A5A68B2FBF0F600FB16228AB918683A
:10298000DA6890420DD2121AC3E90024302383F38F
:10299000118821462846FFF78BFF84F31188BDE894
:1029A000F081012303FA04F26B8923EA02036B81AD
:1029B000CB68002BF3D021462846BDE8F0411847EC
:1029C00000EB81034A0170B5DD68D0F890306C6986
:1029D0002668E66056BB1A444FF40020C2F810097E
:1029E0002A6802F00302012A0AB20ED1D3F80808BD
:1029F00003EB421410F4807FD4F8000914BF40F0B8
:102A0000805040F00050C4F8000903EB4212D2F8A5
:102A1000000940F00440C2F800090122D3F834084C
:102A200002FA01F10143C3F8341870BD19B9402E00
:102A300084BF4020206020681A442E8A8419013CFB
:102A4000B4FBF6F440EAC44040F00050C6E7000092
:102A50002DE9F843D0F8906005460C464F0106EB8F
:102A60004113D3F8088918F0010FC3F808891CD066
:102A7000D6F81038DB0718D500EB8103D3F80CC06B
:102A8000DCF81430D3F800E0DA68964530D2A2EBD7
:102A90000E024FF000091A60C3F80490302383F34C
:102AA0001188FFF78DFF89F3118818F0800F1DD072
:102AB000D6F834380126A640334217D005EB8403FC
:102AC0000134D5F89050D3F80CC0E4B22F44DCF8B0
:102AD000142005EB0434D2F800E05168714514D39A
:102AE000D5F8343823EA0606C5F83468BDE8F8831B
:102AF000012303FA01F2038923EA02030381DCF8CC
:102B00000830002BD1D09847CFE7AEEB0103BCF8DB
:102B10001000834228BF0346D7F8180980B2B3EBF0
:102B2000800FE3D89068A0F1040959F8048FC4F825
:102B30000080A0EB09089844B8F1040FF5D81844B8
:102B40000B4490605360C8E72DE9F84FD0F89050DF
:102B500004466E69AB691E4016F480586E6103D05E
:102B6000BDE8F84FFEF730BC002E12DAD5F8003E73
:102B70009B0705D0D5F8003E23F00303C5F8003EBF
:102B8000D5F80438204623F00103C5F80438FEF7D1
:102B900049FC370505D52046FFF772FC2046FEF7B5
:102BA0002FFCB0040CD5D5F8083813F0060FEB68ED
:102BB00023F470530CBF43F4105343F4A053EB6061
:102BC00031071BD56368DB681BB9AB6923F00803C9
:102BD000AB612378052B0CD1D5F8003E9A0705D0C0
:102BE000D5F8003E23F00303C5F8003E2046FEF76B
:102BF00019FC6368DB680BB120469847F30200F1CB
:102C0000BA80B70226D5D4F8909000274FF0010A79
:102C100009EB4712D2F8003B03F44023B3F5802FB1
:102C200011D1D2F8003B002B0DDA62890AFA07F3C2
:102C300022EA0303638104EB8703DB68DB6813B1DB
:102C40003946204698470137D4F89430FFB29B6844
:102C50009F42DDD9F00619D5D4F89000026AC2F37C
:102C60000A1702F00F0302F4F012B2F5802F00F001
:102C7000CA80B2F5402F09D104EB8303002200F58E
:102C80008050DB681B6A974240F0B0803003D5F873
:102C9000185835D5E90303D500212046FFF746FE35
:102CA000AA0303D501212046FFF740FE6B0303D59D
:102CB00002212046FFF73AFE2F0303D503212046C9
:102CC000FFF734FEE80203D504212046FFF72EFE6D
:102CD000A90203D505212046FFF728FE6A0203D585
:102CE00006212046FFF722FE2B0203D507212046AE
:102CF000FFF71CFEEF0103D508212046FFF716FE63
:102D0000700340F1A780E90703D500212046FFF7B3
:102D10009FFEAA0703D501212046FFF799FE6B0706
:102D200003D502212046FFF793FE2F0703D5032189
:102D30002046FFF78DFEEE0603D504212046FFF75F
:102D400087FEA80603D505212046FFF781FE690608
:102D500003D506212046FFF77BFE2A0603D507216F
:102D60002046FFF775FEEB0574D520460821BDE827
:102D7000F84FFFF76DBED4F890904FF0000B4FF076
:102D8000010AD4F894305FFA8BF79B689F423FF6B4
:102D900038AF09EB4713D3F8002902F44022B2F50B
:102DA000802F20D1D3F80029002A1CDAD3F800297B
:102DB00042F09042C3F80029D3F80029002AFBDB37
:102DC0003946D4F89000FFF787FB22890AFA07F307
:102DD00022EA0303238104EB8703DB689B6813B1BA
:102DE0003946204698470BF1010BCAE7910701D1FC
:102DF000D0F80080072A02F101029CBF03F8018B82
:102E00004FEA18283FE704EB830300F58050DA68A7
:102E1000D2F818C0DCF80820DCE9001CA1EB0C0C8F
:102E200000218F4208D1DB689B699A683A449A6016
:102E30005A683A445A6029E711F0030F01D1D0F8DB
:102E400000808C4501F1010184BF02F8018B4FEA3B
:102E50001828E6E7BDE8F88F08B50348FFF774FEC9
:102E6000BDE8084000F07ABB6441002008B5034883
:102E7000FFF76AFEBDE8084000F070BB004200208A
:102E8000D0F8903003EB4111D1F8003B43F400132C
:102E9000C1F8003B70470000D0F8903003EB4111BF
:102EA000D1F8003943F40013C1F80039704700002D
:102EB000D0F8903003EB4111D1F8003B23F400131C
:102EC000C1F8003B70470000D0F8903003EB41118F
:102ED000D1F8003923F40013C1F80039704700001D
:102EE000090100F16043012203F56143C9B283F88F
:102EF000001300F01F039A4043099B0003F1604355
:102F000003F56143C3F880211A60704730B504337C
:102F1000039C0172002104FB0325C160C0E9065334
:102F2000049B0363059BC0E90000C0E90422C0E9DB
:102F30000842C0E90A11436330BD00000022416A23
:102F4000C260C0E90411C0E90A226FF00101FEF776
:102F500099BD0000D0E90432934201D1C2680AB998
:102F6000181D704700207047036919600021C2686E
:102F70000132C260C269134482699342036124BF73
:102F8000436A0361FEF772BD38B504460D46E36837
:102F90003BB162690020131D1268A3621344E3620F
:102FA00007E0237A33B929462046FEF74FFD002873
:102FB000EDDA38BD6FF00100FBE70000C368C269BD
:102FC000013BC3604369134482699342436124BF58
:102FD000436A436100238362036B03B11847704760
:102FE00070B53023044683F31188866A3EB9FFF733
:102FF000CBFF054618B186F31188284670BDA36A39
:10300000E26A13F8015B9342A36202D32046FFF702
:10301000D5FF002383F31188EFE700002DE9F84F77
:1030200004460E46174698464FF0300989F311883A
:103030000025AA46D4F828B0BBF1000F09D14146BB
:103040002046FFF7A1FF20B18BF311882846BDE889
:10305000F88FD4E90A12A7EB050B521A934528BF43
:103060009346BBF1400F1BD9334601F1400251F8A2
:10307000040B914243F8040BF9D1A36A4036403562
:103080004033A362D4E90A239A4202D32046FFF7D1
:1030900095FF8AF31188BD42D8D289F31188C9E718
:1030A00030465A46FDF7BAFEA36A5E445D445B446F
:1030B000A362E7E710B5029C0433017203FB04210D
:1030C000C460C0E906130023C0E90A33039B03630D
:1030D000049BC0E90000C0E90422C0E90842436340
:1030E00010BD0000026A6FF00101C260426AC0E9CF
:1030F00004220022C0E90A22FEF7C4BCD0E904235E
:103100009A4201D1C26822B9184650F8043B0B60BC
:10311000704700231846FAE7C3680021C2690133EB
:10312000C3604369134482699342436124BF436A85
:103130004361FEF79BBC000038B504460D46E368CA
:103140003BB1236900201A1DA262E2691344E362C5
:1031500007E0237A33B929462046FEF777FC00289A
:10316000EDDA38BD6FF00100FBE70000036919607C
:10317000C268013AC260C269134482699342036122
:1031800024BF436A036100238362036B03B11847C2
:103190007047000070B530230D460446114683F396
:1031A0001188866A2EB9FFF7C7FF10B186F3118820
:1031B00070BDA36A1D70A36AE26A01339342A362E1
:1031C00004D3E16920460439FFF7D0FF002080F3E3
:1031D0001188EDE72DE9F84F04460D4690469946D3
:1031E0004FF0300A8AF311880026B346A76A4FB918
:1031F00049462046FFF7A0FF20B187F311883046EB
:10320000BDE8F88FD4E90A073A1AA8EB06079742F7
:1032100028BF1746402F1BD905F1400355F8042B52
:103220009D4240F8042BF9D1A36A40364033A36293
:10323000D4E90A239A4204D3E16920460439FFF70E
:1032400095FF8BF311884645D9D28AF31188CDE7D3
:1032500029463A46FDF7E2FDA36A3D443E443B441D
:10326000A362E5E7D0E904239A4217D1C3689BB172
:10327000836A8BB1043B9B1A0ED01360C368013B79
:10328000C360C3691A4483699A42026124BF436AD6
:103290000361002383620123184670470023FBE784
:1032A00000F086B9014B586A704700BF000C00401F
:1032B000034B002258631A610222DA60704700BF94
:1032C000000C0040014B0022DA607047000C004007
:1032D000014B5863704700BF000C0040FEE7000040
:1032E00070B51B4B0025044686B058600E468562BB
:1032F000016300F00BF904F11003A560E562C4E975
:1033000004334FF0FF33C4E90044C4E90635FFF746
:10331000C9FF2B46024604F134012046C4E90823C4
:1033200080230C4A2565FEF747FB01230A4AE0602B
:1033300000920375684672680192B268CDE9022373
:10334000064BCDE90435FEF75FFB06B070BD00BF4C
:1033500020260020243D0008293D0008DD32000819
:10336000024AD36A1843D062704700BFB8230020D6
:103370004B6843608B688360CB68C3600B694361B3
:103380004B6903628B6943620B68036070470000FE
:1033900008B53C4B40F2FF713B48D3F888200A4304
:1033A000C3F88820D3F8882022F4FF6222F00702B5
:1033B000C3F88820D3F88820D3F8E0200A43C3F864
:1033C000E020D3F808210A43C3F808212F4AD3F894
:1033D00008311146FFF7CCFF00F5806002F11C01B7
:1033E000FFF7C6FF00F5806002F13801FFF7C0FF6C
:1033F00000F5806002F15401FFF7BAFF00F580602C
:1034000002F17001FFF7B4FF00F5806002F18C015A
:10341000FFF7AEFF00F5806002F1A801FFF7A8FFFB
:1034200000F5806002F1C401FFF7A2FF00F58060A3
:1034300002F1E001FFF79CFF00F5806002F1FC0162
:10344000FFF796FF02F58C7100F58060FFF790FFA3
:1034500000F076F90E4BD3F8902242F00102C3F847
:103460009022D3F8942242F00102C3F8942205225C
:10347000C3F898204FF06052C3F89C20054AC3F867
:10348000A02008BD0044025800000258303D00084A
:1034900000ED00E01F00080308B500F025FBFEF773
:1034A0004FFA0F4BD3F8DC2042F04002C3F8DC2087
:1034B000D3F8042122F04002C3F80421D3F80431E8
:1034C000084B1A6842F008021A601A6842F00402B7
:1034D0001A60FEF721FFBDE80840FEF7BFBC00BF41
:1034E000004402580018024870470000EFF30983B7
:1034F000054968334A6B22F001024A6383F3098865
:10350000002383F31188704700EF00E0302080F340
:10351000118862B60D4B0E4AD96821F4E0610904A6
:10352000090C0A430B49DA60D3F8FC2042F08072A0
:10353000C3F8FC20084AC2F8B01F116841F001012D
:1035400011602022DA7783F82200704700ED00E056
:103550000003FA0555CEACC5001000E0302310B5CD
:1035600083F311880E4B5B6813F4006314D0F1EE03
:10357000103AEFF309844FF08073683CE361094B24
:10358000DB6B236684F30988FEF7AEF910B1064BB6
:10359000A36110BD054BFBE783F31188F9E700BF7A
:1035A00000ED00E000EF00E02F0400083204000806
:1035B000114BD3F8E82042F00802C3F8E820D3F812
:1035C000102142F00802C3F810210C4AD3F8103140
:1035D000D36B43F00803D363C722094B9A624FF0C1
:1035E000FF32DA6200229A615A63DA605A6001227D
:1035F0005A611A60704700BF004402580010005C16
:10360000000C0040094A08B51169D3680B40D9B2D3
:103610009B076FEA0101116107D5302383F31188FD
:10362000FEF7A4F9002383F3118808BD000C0040C5
:10363000064BD3F8DC200243C3F8DC20D3F8042186
:103640001043C3F80401D3F8043170470044025812
:103650003A4B4FF0FF31D3F8802062F00042C3F8BC
:103660008020D3F8802002F00042C3F88020D3F8F5
:103670008020D3F88420C3F88410D3F8842000225B
:10368000C3F88420D3F88400D86F40F0FF4040F4A2
:10369000FF0040F4DF4040F07F00D867D86F20F093
:1036A000FF4020F4FF0020F4DF4020F07F00D867C7
:1036B000D86FD3F888006FEA40506FEA5050C3F8D3
:1036C0008800D3F88800C0F30A00C3F88800D3F854
:1036D0008800D3F89000C3F89010D3F89000C3F896
:1036E0009020D3F89000D3F89400C3F89410D3F846
:1036F0009400C3F89420D3F89400D3F89800C3F84A
:103700009810D3F89800C3F89820D3F89800D3F80D
:103710008C00C3F88C10D3F88C00C3F88C20D3F83D
:103720008C00D3F89C00C3F89C10D3F89C10C3F80D
:103730009C20D3F89C3000F0AFB900BF0044025881
:1037400008B50122534BC3F80821534BD3F8F4209A
:1037500042F00202C3F8F420D3F81C2142F0020226
:10376000C3F81C210222D3F81C314C4BDA605A6892
:103770009104FCD54A4A1A6001229A60494ADA60EB
:1037800000221A614FF440429A61444B9A699204B4
:10379000FCD51A6842F480721A603F4B1A6F12F41B
:1037A000407F04D04FF480321A6700221A671A68EB
:1037B00042F001021A60384B1A685007FCD500220B
:1037C0001A611A6912F03802FBD1012119604FF019
:1037D000804159605A67344ADA62344A1A611A6879
:1037E00042F480321A602C4B1A689103FCD51A6897
:1037F00042F480521A601A689204FCD52C4A2D4972
:103800009A6200225A63196301F57C01DA6301F2BE
:10381000E71199635A64284A1A64284ADA621A68D6
:1038200042F0A8521A601C4B1A6802F02852B2F1FA
:10383000285FF9D148229A614FF48862DA61402208
:103840001A621F4ADA641F4A1A651F4A5A651F4ADC
:103850009A6532231E4A1360136803F00F03022B8C
:10386000FAD10D4A136943F003031361136903F09E
:103870003803182BFAD14FF00050FFF7D9FE4FF064
:103880008040FFF7D5FE4FF00040BDE80840FFF74D
:10389000CFBE00BF008000510044025800480258CB
:1038A00000C000F0020000010000FF010088900845
:1038B0001210200063020901470E0508DD0BBF014D
:1038C00020000020000001100910E000000101109C
:1038D000002000524FF0B04208B5D2F8883003F013
:1038E0000103C2F8883023B1044A13680BB1506851
:1038F0009847BDE80840FFF731BE00BFB442002042
:103900004FF0B04208B5D2F8883003F00203C2F895
:10391000883023B1044A93680BB1D0689847BDE85A
:103920000840FFF71BBE00BFB44200204FF0B0427A
:1039300008B5D2F8883003F00403C2F8883023B108
:10394000044A13690BB150699847BDE80840FFF776
:1039500005BE00BFB44200204FF0B04208B5D2F817
:10396000883003F00803C2F8883023B1044A936911
:103970000BB1D0699847BDE80840FFF7EFBD00BF25
:10398000B44200204FF0B04208B5D2F8883003F0BE
:103990001003C2F8883023B1044A136A0BB1506A8D
:1039A0009847BDE80840FFF7D9BD00BFB4420020EA
:1039B0004FF0B04310B5D3F8884004F47872C3F8E0
:1039C0008820A30604D5124A936A0BB1D06A98479F
:1039D000600604D50E4A136B0BB1506B9847210655
:1039E00004D50B4A936B0BB1D06B9847E20504D515
:1039F000074A136C0BB1506C9847A30504D5044AD1
:103A0000936C0BB1D06C9847BDE81040FFF7A6BD92
:103A1000B44200204FF0B04310B5D3F8884004F40E
:103A20007C42C3F88820620504D5164A136D0BB199
:103A3000506D9847230504D5124A936D0BB1D06D94
:103A40009847E00404D50F4A136E0BB1506E9847A7
:103A5000A10404D50B4A936E0BB1D06E9847620453
:103A600004D5084A136F0BB1506F9847230404D54F
:103A7000044A936F0BB1D06F9847BDE81040FFF731
:103A80006DBD00BFB442002008B5FFF7BBFDBDE827
:103A90000840FFF763BD0000062108B50846FFF7A0
:103AA0001FFA06210720FFF71BFA06210820FFF75F
:103AB00017FA06210920FFF713FA06210A20FFF75B
:103AC0000FFA06211720FFF70BFA06212820FFF72F
:103AD00007FA09217A20FFF703FA07213220BDE80F
:103AE0000840FFF7FDB9000008B5FFF7B1FD00F091
:103AF0000BF8FDF7F7FBFDF7C9FAFFF7F5FCBDE89A
:103B00000840FFF7CDBB00000023054A19460133EA
:103B1000102BC2E9001102F10802F8D1704700BF72
:103B2000B442002010B501390244904201D1002076
:103B300005E0037811F8014FA34201D0181B10BD16
:103B40000130F2E7034611F8012B03F8012B002A9C
:103B5000F9D1704753544D333248373F3F3F0053FC
:103B6000544D3332483733782F3732780053544D21
:103B70003332483734332F3735332F373530000061
:103B800001105A000310590001205800032056006C
:103B90000000000009100008F50F000831100008AF
:103BA0001D10000829100008151000080110000859
:103BB000ED0F00083D1000080000000001000000AB
:103BC0000000000063300000C43B00081024002007
:103BD000202600204172647550696C6F7400254284
:103BE0004F415244252D424C002553455249414CEA
:103BF000250000000200000000000000291200085B
:103C00009912000840004000D03E0020E03E002015
:103C1000020000000000000003000000000000009F
:103C2000E11200080000000010000000F03E00203B
:103C300000000000010000000000000064410020BE
:103C400001010200F91D0008091D0008A51D00085A
:103C5000891D0008430000005C3C00080902430085
:103C6000020100C032090400000102020100052423
:103C700000100105240100010424020205240600AD
:103C800001070582030800FF09040100020A000081
:103C90000007050102400000070581024000000006
:103CA00012000000A83C00081201100102000040B0
:103CB0000912415700020102030100000403090434
:103CC00025424F415244250053444D4F44454C48F2
:103CD0003756310030313233343536373839414296
:103CE0004344454600000000000000003D14000869
:103CF000F5160008A1170008400040009C42002073
:103D00009C42002001000000AC4200208000000026
:103D10004001000008000000000100000010000049
:103D2000080000006D61696E0069646C6500000048
:103D30000001802A00000000AAAAAAAA000100240B
:103D4000FFFF00000000000000A00A00000040018A
:103D500000000000AAAAAAAA00000001FFFF0000BC
:103D6000000000000000000010000004000000003F
:103D7000AAAAAAAA00000008FBDF000000000000B9
:103D8000000000000000000000000000AAAAAAAA8B
:103D900000000000FFFF0000000000000000000025
:103DA0000001000000000000AAAAAAAA0001000069
:103DB000FFFF000000000000000000000000000005
:103DC00000000000AAAAAAAA00000000FFFF00004D
:103DD00000000000000000000000000000000000E3
:103DE000AAAAAAAA00000000FFFF0000000000002D
:103DF000000000000000000000000000AAAAAAAA1B
:103E000000000000FFFF00000000000000000000B4
:103E10000000000000000000AAAAAAAA00000000FA
:103E2000FFFF000000000000000000000000000094
:103E300000000000AAAAAAAA00000000FFFF0000DC
:103E40000000000000000000000000000000000072
:103E5000AAAAAAAA00000000FFFF000000000000BC
:103E600000000000000000005704000000000000F7
:103E700000001A0000000000FF0000000000000029
:103E8000543B0008830400005F3B0008500400001E
:103E90006D3B00080096000000000800960000003E
:103EA0000008000004000000BC3C00080000000006
:103EB0000000000000000000000000000000000002
:043EC00000000000FE
:00000001FF
